:020000040000FA
:10000000E029FF3FFF3FFF3FF000030EF10004082F
:10001000F2000A08F30083018A018C184F290C189A
:10002000FD288B1857290B1918288C1A66291728B0
:1000300083010B11311E2C28061DCC01CC0A4C0863
:10004000123C031D412831124015C0107027CC010D
:100050000A30C900E40141280619CB01CB0A4B083C
:10006000183C031D41283116CB01DE10E301C111FC
:1000700041124015311F4128C0144011AE270A30EB
:10008000C9003608031D4A28311D5528861009303D
:10009000B6005528B60B4F28861431115528B70CD9
:1000A000031C86100318861455283F0803195A2884
:1000B000BF037B2831197B28BD1F66283D086925B1
:1000C000B7003115BD010C30BF007B28BE1F702862
:1000D0003E086925B7003115BE010C30BF007B28F2
:1000E000411D7B2841110330BC006925B700311543
:1000F000BE010C30BF003B0803198028BB039328C6
:100100000C1E9328B91F8B28390869259900B9015D
:100110003230BB009328BA1F93283A08692599000A
:10012000BA013230BB0049080319B728C90349088E
:10013000FC39031DB7288A01490803398207A3281F
:10014000AB28B028B42807153C30DD0007160000A6
:1001500007128C11B7288C110310480D9300B72893
:100160008C1147089300B7288C11460893004D085E
:100170000319C628CD0BBF2806128616C6284D1CAB
:10018000C42806168616C62806128612411FCB28DA
:100190004113803091005D080319D128DD0BD1286F
:1001A00007118301E208031D6400E10BFC2878308D
:1001B000E100E208031DE2035F080319E228DF0BF8
:1001C000E228C11460080319E828E00BE82841146C
:1001D0006408031DED281211EE28E40363080319D7
:1001E000FC28E30BF82840153C30CD004112FC28D8
:1001F0006308073903194116D72983010C10F03021
:1002000010108F0710140314061C0310B20B4C2996
:10021000031C4729B41B472933084D25B11D472925
:10022000B500B1143C02031D18298030BC004629DA
:100230003508F039403C031942293508F039503C63
:10024000031942293508F039603C03194229350861
:10025000F039303C031933293508763C031D322927
:10026000B116332946294E0A57395038CE0084003A
:1002700035088000C117313C03193113FC3C0319C8
:10028000311742293508BC00BD00BD170000101011
:100290000C100B168B104E29B30CB40CD72983010C
:1002A0008C10861D5529861156298615D72983015C
:1002B0008B100B1E13289001FC308F0020308E0015
:1002C0000C100B1210140A30B200D72983019818B1
:1002D000D2291819D2291A084D25B11DD129A600F5
:1002E0003802031D76298030B800D6292608F03957
:1002F000031D8329B11E7E29B1128229311A822958
:100300003C30CD00882926087E3C031988298B299A
:100310002608B900B9177E302602031D9129C0179F
:10032000D6292608F039031DD629C01BD629630813
:1003300003199F29E301C11141124015C429083056
:100340002602031DA5294017D62907302602031DC2
:10035000AB29C016D62906302602031DB129401646
:10036000D62905302602031DB729C015D629043029
:100370002602031DC429311EC229311FC32941177A
:100380004014C329C115D629033026020319CC29EC
:1003900000302602031DD0292608BC00BE00BE176F
:1003A000D629D6291A081A0818121816D729730838
:1003B0008A0072088400710E8300F00E700E09002E
:1003C00083018A018B0164000030850023308600A0
:1003D000C4308700831683308100C130850005302A
:1003E0008600803087008312830181309F0083164E
:1003F0008E309F0083010030900083018316AF3060
:10040000920083013830920097019D0183010230F0
:10041000940083164030940083129416830183164F
:10042000FF309900203098008301903098008301BC
:10043000B101DE01B201B301B401B501B601B701EA
:10044000B901BA018030B8003230BB00BD01BE0135
:100450008030BC000C30BF00C001C017C10150305B
:10046000CE00CF00C401C901CA01CD01DD01DF0109
:10047000E001E301E4017830E1001E30E2000030E9
:100480005F25C2009F3C0318472A7830C200013024
:100490005F25C300013043020319582A023043028A
:1004A0000319582A083043020319582A0230C3009E
:1004B0003030C50070271225071183018C018D0192
:1004C000831623308C008D0183018B01F0308B006B
:1004D00083011E30E200C11BB82AC01B862B8B1380
:1004E000311E762A4013C012C0114012C018CA2A09
:1004F0004019FB2A40182A2BC119302B411A652BB1
:10050000401B682CC01A7C2CC019FF2B401AE72C0A
:10051000C1188E2A4118A42A8B17682A42085E182F
:10052000450703178C0000308D0083168C010C15D5
:1005300055308D00AA308D008C148B138C189E2A98
:100540000C118301C110682A430803178C00013085
:100550008D0083168C010C1555308D00AA308D004E
:100560008C148B138C18B22A0C1183014110682A49
:100570008B134F0884004E020319C72A4F0A5739BC
:100580005038CF00840000088B173625B82AC113D5
:100590008B17682A8B17AC0142084407AB00031085
:1005A0002C308400D42542084407B000AF012C3021
:1005B000A7003030A800FD252C30A7003030A8005F
:1005C000FD252C30A7003030A800FD257A256130AC
:1005D00036256130362541303625443036255808D9
:1005E0003625590836255A0836255B0836255C0815
:1005F0003625C010682A8B17AC014208AB000310E7
:100600002C308400D4254208B000AF012C30A70064
:100610003030A800FD252C30A7003030A800FD2583
:100620002C30A7003030A800FD257A256130362512
:100630006130362541303625443036255808362578
:10064000590836255A0836255B0836255C083625B4
:100650004011682A8B170A30E40012154010682AEE
:100660006430E3008B1761303625613036254C301D
:1006700036254C3036254C3036254C3036254C301E
:1006800036254C3036254C30362583011F150000A9
:100690001F19482B83161E088301AC001E08AB00EF
:1006A0002C3084000310D4252C3084000310D42572
:1006B0007A2562303625623036255A0836255B08A1
:1006C00036255C083625C111682A8B1783011F1552
:1006D00000001F19692B83161E088301AC001E0839
:1006E000AB002C3084000310D4252C308400031080
:1006F000D4257A2562303625623036255A083625CB
:100700005B0836255C0836254112682A1C261C2603
:100710001C261C261C26AC014208AB0003102C3002
:100720008400D4254208B000AF012C30A70030303F
:10073000A800FD252C30A7003030A800FD252C3066
:10074000A7003030A800FD257A25603036254C30D2
:100750003625613036254130362562303625443025
:100760003625633036255808362564303625590835
:100770003625653036255A083625663036255B081D
:100780003625673036255C0836254508303C031D84
:10079000D42B80304202031CD42B42088F3C031C14
:1007A000D42BD030C400D62BC401DD2B60303625CD
:1007B0006D3036256E303625E32B603036256D30B2
:1007C00036256D3036256D3036256D3036256D3049
:1007D0003625083043026D3003196E30362502305D
:1007E00043026D3003196E303625013043026D30FF
:1007F00003196E303625311F4115C013682A44088D
:100800000319182CC41F202CDE18322CDE145E14A1
:100810004508C400C20270270A30C9007830CA00F7
:100820008B17603036256E3036256D303625402CDE
:100830004508003CC4004207A03C031C322C242C79
:100840004508C207003CC4005E1070270A30C9008A
:100850007830CA008B17603036256D3036256E3003
:100860003625402CDE10C40170270A30C9007830CC
:10087000CA008B17603036256D3036256D30362531
:10088000AC014208AB0003102C308400D425420890
:10089000B000AF012C30A7003030A800FD252C306F
:1008A000A7003030A800FD252C30A7003030A8006C
:1008B000FD257A2563303625580836255908362512
:1008C0005A0836255B0836255C083625C011682A8B
:1008D0005E1C6D2C5E104508C20742084307C2002B
:1008E0004308013C031D421042089F3C03187A2C28
:1008F000A030C2024013922C5E1C812C5E10450871
:10090000C20743084202C2004308013C03198A2C73
:100910004218C20A4208A03C0318902CA030C2071B
:10092000C012922C70270A30C9007830CA00DE103D
:100930008B173230DF00AC014208AB0003102C30C3
:100940008400D4254208B000AF012C30A70030301D
:10095000A800FD252C30A7003030A800FD252C3044
:10096000A7003030A800FD257A25633036255808C9
:100970003625590836255A0836255B0836255C0881
:1009800036254508303C031DD42C80304202031C20
:10099000D42C42088F3C031CD42C4408D03C0319AF
:1009A000E62CD030C400D92C44080319E62CC4012D
:1009B000E02C603036256D3036256E303625E62C3D
:1009C000603036256D3036256D303625682A8B1718
:1009D0003230E0004308023C031DF72C0830C3000E
:1009E000653036256E3036256D303625102D43089E
:1009F000083C031D062D0130C300653036256D30DF
:100A000036256D3036256E303625102D0230C30068
:100A1000653036256D3036256E3036256D303625FD
:100A20004012682A830107128C11123093008C1D2A
:100A3000172D8C11013093008C1D1C2D0716000002
:100A400007128C11460893008C1D242D8C11470829
:100A500093008C1D292D8C110310480D93008C1DC3
:100A60002F2D0716000007128C1108008301A0002B
:100A7000BA1B382D7F39B800BA00BA17FA30A10076
:100A8000F530A30000000000A30B422DB81B4C2D35
:100A9000A10B402D2008382D08008301B111A400BE
:100AA000A500240E2406A400A40D2406A40D2406EB
:100AB000A40DA406A41BB1157F30250508008301F1
:100AC00003178D0083168C010C1483120C0883010C
:100AD000080083017F39A400A500240E2406A40089
:100AE000A40D2406A40D2406A40D2406803A803902
:100AF000250408001030B0002730AF00FF30A300FD
:100B0000A30A2C30A7003030A800FD250318802D43
:100B10002C30A7003030A800E1252308443ED8003F
:100B2000E830B0000330AF00FF30A300A30A2C3040
:100B3000A7003030A800FD250318962D2C30A70003
:100B40003030A800E1252308403ED9006430B000D1
:100B5000AF01FF30A300A30A2C30A7003030A8005B
:100B6000FD250318AB2D2C30A7003030A800E1255F
:100B70002308403EDA000A30B000AF01FF30A30086
:100B8000A30A2C30A7003030A800FD250318C02D83
:100B90002C30A7003030A800E1252308403EDB00C0
:100BA0002C08403EDC0008008403DD2D8403840310
:100BB0008403800C840A800C840A800C840A800CD4
:100BC00008000230A2000310E82D0430A200031038
:100BD000280884000008A1002708840003110318D6
:100BE000800A3110031931142108800731180314C9
:100BF000A703A803A20BE82D08000230A2000314EB
:100C0000042E0430A2000314280884000008A10068
:100C100027088400031C0E2E3110132E800831107B
:100C20000319311480032108800231180310A7032F
:100C3000A803A20B042E0800C830A000F530A100C4
:100C40000000000000000000000000000000A10BF8
:100C5000202EA00B1E2E08002830A000F530A10089
:100C600000000000A10B302EA00B2E2E0800F53046
:100C7000A0000000000000000000000000000000D4
:100C80000000000000000000000000000000000064
:100C900000000000A00B392E0800FF3FFF3FFF3F80
:100CA000FF3FFF3FFF3FFF3FFF3FFF3FFF3FFF3F54
:100CB000FF3FFF3FFF3FFF3FFF3FFF3FFF3FFF3F44
:100CC000FF3FFF3FFF3FFF3FFF3FFF3FFF3FFF3F34
:100CD000FF3FFF3FFF3FFF3FFF3FFF3FFF3FFF3F24
:100EE00007308A00420EC800480C073982077F2F5E
:100EF000882F912F9A2FA32FAC2FAC2FAC2F01301E
:100F0000C600EA30C700420D3E39103EC800AD2F82
:100F10000130C600EC30C700420D3E39003EC8002B
:100F2000AD2F0130C600ED30C700420D3E39183EEE
:100F3000C800AD2F0130C600EF30C700420D3E396A
:100F4000083EC800AD2F0130C600F030C700420D8A
:100F50003E39203EC800AD2FAC2F080007308A0074
:100F600044084207C800480EC800480C07398207E9
:100F7000C02FCC2FD82FE42FF02FFC2FFC2FFC2FCD
:100F80000230C6004030C70042084407C800480D80
:100F90003E39003EC800FD2F0230C6004130C70078
:100FA00042084407C800480D3E39183EC800FD2FCE
:100FB0000230C6004330C70042084407C800480D4D
:100FC0003E39083EC800FD2F0230C6004430C7003D
:100FD00042084407C800480D3E39203EC800FD2F96
:100FE0000230C6004630C70042084407C800480D1A
:100FF0003E39103EC800FD2FFC2F0800FF3FFF3F89
:10100000FF3FFF3FFF3FFF3FFF3FFF3FFF3FFF3FF0
:10101000FF3FFF3FFF3FFF3FFF3FFF3FFF3FFF3FE0
:10102000FF3FFF3FFF3FFF3FFF3FFF3FFF3FFF3FD0
:10103000FF3FFF3FFF3FFF3FFF3FFF3FFF3FFF3FC0
:084000000200120001007F0024
:02400E00763DFD
:00000001FF
